:0400000039EF10F0D4
:1000080000C016F001C015F0E1CF17F0E2CF18F0EC
:100018009EAA47D09DAA45D0ACA203D0AC98AC8884
:10002800AC92ACA402D0AFCF3CF0D6EC0BF000C041
:100038003CF000500D0A08E0000E0001965D02E158
:10004800800E955D01E21FD00001010E3D6E000E8D
:100058003E6E000E965D02E1800E955D04E3020E91
:100068003D6E000E3E6EA09AC80E9525E16E000EFC
:100078009621E26EE66A95C03AF096C03BF0956B21
:10008800966B3C6A0ED0C80E9525E16E000E96213F
:10009800E26E3CC0E6FF95C03AF096C03BF0954B47
:1000A800962BA4AA55D0A3AA53D09CA203D09C985F
:1000B8009C889C929CA404D0AACF2CF202012C6BA1
:1000C8000201AACF2CF22C510A0A14E1010E0001F8
:1000D8008F6F000E906F5F0E9125E16E020E9221D8
:1000E800E26E2CC2E6FF91C093F092C094F0020138
:1000F8002C6B0FD05F0E00019125E16E020E92214C
:10010800E26E2CC2E6FF91C093F092C094F0914B3E
:10011800922B0001000E925D02E1800E915D18E3C2
:10012800020E8F6F000E906FA09A010E915F000E65
:10013800925B5F0E9125E16E020E9221E26EE66AF5
:1001480091C093F092C094F0916B926B02012C6B6A
:10015800F2AA16D0F2A414D00201124B132B000EEF
:10016800006E1351005C02E11251020808E2010E10
:10017800146F000E156FF29A126B136BD59EF294E2
:1001880016C000F015C001F017C0E1FF18C0E2FF6B
:02019800110054
:10019A000B820BAED7EF00F00368026801680068B3
:0801AA000A360232FF0E1200BA
:0E01B200026A016A006A086A036A000E1200FF
:1001C0000B840BAEEBEF00F0010E036E026A016AC6
:0A01D000006A0A360232FF0E120028
:0801DA000AAE029E000E1200A5
:1001E2000CB033EF01F00CA2D9EF01F00E6A000E51
:1001F20002644AEF01F0F00E0214D8A415EF01F0E8
:10020200023A01380F0B02260138F00B016E00385A
:100212000F0B01260038F00B006E08380F0B00267A
:100222000838F00B086E0E84D89002BE2EEF01F053
:1002320008360036013602360E2A02BE2EEF01F0D3
:1002420008360036013602360E2A02BE2EEF01F0C3
:1002520008360036013602360E2A0E500364CFEFFE
:1002620001F0035E0BBC08AED4EF01F0D880800E23
:1002720008640030000E002201220222D8A0D4EF2E
:1002820001F0023201320032034AD9EF01F0D4EF19
:1002920001F001C002F000C001F008C000F0086ADD
:1002A200000E0E86026481EF01F0F00E0214D8A453
:1002B20069EF01F0023A01380F0B02260138F00B08
:1002C200016E00380F0B01260038F00B006E0E8411
:1002D200D89002BE2EEF01F00036013602360E2A09
:1002E20002BE2EEF01F00036013602360E2A02BEA1
:1002F2002EEF01F00036013602360E2A2EEF01F003
:1003020001C002F000C001F0006A000E0E960E88D5
:100312000264AEEF01F0F00E0214D8A499EF01F0DE
:10032200023A01380F0B02260138F00B016E0E84DF
:10033200D89002BE2EEF01F0013602360E2A02BE1E
:100342002EEF01F0013602360E2A02BE2EEF01F028
:10035200013602360E2A2EEF01F001C002F0016AC8
:10036200000E0E860264DEEF01F0F00E0214D8A435
:10037200BDEF01F0023A0E84D89002BE2EEF01F0DA
:1003820002360E2A02BE2EEF01F002360E2A02BEFD
:100392002EEF01F002360E2A2EEF01F0010E0C6E46
:1003A2000EDFE1EF01F0020E0C6E16DFE1EF01F05D
:1003B200040E0C6EF1DEE1EF01F0080E0C6EF8DEB9
:0203C200120027
:1003C4000B800BAEEEEF01F0026A0AAEFF0E026E76
:0C03D400016E006E0A360232FF0E1200AD
:1003E000025006180E6E086A096A0B6A0350076409
:1003F000E3EF02F006500A6E068E028E03500B6E7B
:100400000750036E000E0B6433EF02F00B50075ED3
:10041000D8B4D4EF02F0070E0764A2EF02F0075E33
:1004200000C008F001C000F002C001F0026A074EEF
:10043000D4EF02F0076477EF02F0075E00C008F027
:1004400001C000F0016A074ED4EF02F0076455EFD7
:1004500002F0075E00C008F0006A074ED4EF02F019
:1004600007643CEF02F00AC002F005C001F004C0CE
:1004700000F0086AFDEF03F0030E076447EF02F097
:10048000075E08380F0B086E074ED4EF02F0D890C5
:100490000832074ED4EF02F0D8900832074ED4EF5E
:1004A00002F0D8900832D4EF02F0030E076466EF32
:1004B00002F0075E08380F0B086E0038F00B0826B4
:1004C00000380F0B006E074ED4EF02F0D8900032C8
:1004D0000832074ED4EF02F0D89000320832074EAF
:1004E000D4EF02F0D89000320832D4EF02F0030EBD
:1004F00007648EEF02F0075E08380F0B086E0038B5
:10050000F00B082600380F0B006E0138F00B0026A8
:1005100001380F0B016E074ED4EF02F0D890013274
:1005200000320832074ED4EF02F0D8900132003288
:100530000832074ED4EF02F0D89001320032083270
:10054000D4EF02F0030E0764BFEF02F0075E083835
:100550000F0B086E0038F00B082600380F0B006EEA
:100560000138F00B002601380F0B016E0238F00B3A
:10057000012602380F0B026E074ED4EF02F0D8901E
:100580000232013200320832074ED4EF02F0D89026
:100590000232013200320832074ED4EF02F0D89016
:1005A0000232013200320832096A000E0EAEC8EF84
:1005B00003F0081E001E011E021E082A002201224E
:1005C0000222C8EF03F00750D8A4E9EF02F0FDEFD4
:1005D00003F0096A02C00AF0028E068E0750035C1F
:1005E000076ED8B4BBEF03F0070E076489EF03F082
:1005F000075E0450096E0550046E0650056E066ACB
:10060000074EBBEF03F0070E07645EEF03F0075ED3
:100610000450096E0550046E056A074EBBEF03F0E7
:10062000070E07643CEF03F0075E0450096E046A8E
:10063000074EBBEF03F0070E076423EF03F00AC079
:1006400002F0FDEF03F0030E07642EEF03F0075EE8
:1006500009380F0B096E074EBBEF03F0D890093233
:10066000074EBBEF03F0D8900932074EBBEF03F003
:10067000D8900932BBEF03F0030E07644DEF03F08F
:10068000075E09380F0B096E0438F00B0926043891
:100690000F0B046E074EBBEF03F0D8900432093203
:1006A000074EBBEF03F0D89004320932074EBBEF80
:1006B00003F0D89004320932BBEF03F0030E076455
:1006C00075EF03F0075E09380F0B096E0438F00B65
:1006D000092604380F0B046E0538F00B0426053884
:1006E0000F0B056E074EBBEF03F0D89005320432B6
:1006F0000932074EBBEF03F0D890053204320932BD
:10070000074EBBEF03F0D890053204320932BBEF3D
:1007100003F0030E0764A6EF03F0075E09380F0B22
:10072000096E0438F00B092604380F0B046E0538E7
:10073000F00B042605380F0B056E0638F00B052666
:1007400006380F0B066E074EBBEF03F0D89006324B
:10075000053204320932074EBBEF03F0D89006325F
:10076000053204320932074EBBEF03F0D89006324F
:10077000053204320932086A000E0EAEC8EF03F0EB
:10078000091E041E051E061E092A04220522062231
:10079000095008260450002205500122065002226A
:1007A0000EBEDFEF03F0D8A0EEEF03F0023201320D
:1007B00000320832033EEEEF03F0F8EF03F0D8B05A
:1007C000F3EF03F0000E081E001E011E021E082A91
:1007D0000022012202220A7EF3EF03F0010E0C6ECA
:1007E00000DDFFEF03F0020E0C6EFBDCFFEF03F009
:1007F000040E0C6ED2DCFFEF03F0000E0C6E120044
:100800000C6A0E6A0250D8A419EF04F001C002F07D
:1008100000C001F0006A0E860250D8A419EF04F05F
:1008200001C002F0016A0E960E880250D8B42BEF78
:1008300004F00E50035ED8A4D8A030EF04F0D89096
:1008400002BE35EF04F0003601360236032E20EFEB
:1008500004F030EF04F0010E0C6EABDC38EF04F066
:10086000020E0C6EADDC38EF04F0040E0C6EB5DC3D
:02087000120074
:080872000B6A0B86FF0E120059
:10087A000450000A12E10550000A0FE10650000A6E
:10088A000CE10750000A09E1FF0E006EFF0E016E2F
:10089A007F0E026EFF0E036EA7D0086A096A075020
:1008AA00D8B4E8EF04F00350D8B4ECEF04F00250E7
:1008BA0006180A6E028E068E0E6A02C008F001C081
:1008CA000CF000C00DF004500D5E0550D8A0053C98
:1008DA000C5E0650D8A0063C085E086A0C6A0D6ACF
:1008EA00D8A07FEF04F0D8900232013200320832E9
:1008FA00010E0E6E0750035ED8A08CEF04F07E0E38
:10090A000E240326D8B0F1EF04F092EF04F07E0E25
:10091A000E240326D8A0F6EF04F0180E0B6E0D363F
:10092A000C3608360036013602360E360450005EA2
:10093A000550D8A0053C015E0650D8A0063C025ED0
:10094A0006340E120EA0ADEF04F00D80B8EF04F0DD
:10095A00045000260550D8B0053C01260650D8B0F0
:10096A00062802260D900B2E94EF04F0DEEF04F019
:10097A00D8900036013602360E360450005E055015
:10098A00D8A0053C015E0650D8A0063C025E06349B
:10099A000E10010B0D26D8B00C2AD8B4082AD8A4F8
:1009AA00DEEF04F008320C320D32032AD8B4F1EF2C
:1009BA0004F00AAE089E0850026E0C50016E0D50EB
:1009CA00006EF9EF04F0010E4FDFF9EF04F0020EAA
:1009DA00D9EC00F0F9EF04F0040ECDEC00F0F9EFD9
:0A09EA0004F0080EE0EC00F012002B
:1009F400086A096A000E076203647FEF05F002507B
:100A040006180A6E075003267E0ED8A010EF05F0D4
:100A1400035ED8B084EF05F014EF05F0035ED8A0B0
:100A240089EF05F0028E068E02C00EF001C00BF0B5
:100A340000C00DF000500402F4CF0CF00150050288
:100A4400F4CF00F0F3CF08F00402F3500C26F45076
:100A54000822000E00220D500502F3500C26F4501B
:100A64000822000E002202500402F3500826F4501B
:100A7400002202500502016A000E0122F3500026F2
:100A8400F45001220D500602F3500826F4500022BF
:100A9400026A000E012202220B500602F3500026C5
:100AA400F4500122000E02220E500602F3500126D9
:100AB400F450022202BE67EF05F008360036013614
:100AC40002360306D8B489EF05F07AEF05F0D88032
:100AD400800E08640030000E002201220222D8A0F9
:100AE4007AEF05F0023201320032034A84EF05F056
:100AF4000AAE029E000E8CEF05F0010ED9EC00F058
:100B04008CEF05F0020ECDEC00F08CEF05F0040E36
:060B1400E0EC00F012000D
:0E0B1A00ADB202D00000FCD724C3AEFF120023
:100B2800086A096A100E0C6E01340836093604503A
:100B3800085E0550D8A0053C095ED8B007D004501F
:100B480008260550D8B0053C0926D890003601364D
:060B58000C2EEAD712008A
:0E0B5E00570E0D6E0D2EFED700000000120087
:100B6C0024C3E9FF25C3EAFFEE500301261905E172
:100B7C0024C300F025C301F010D024C300F025C31A
:100B8C0001F0244B252B00C0E9FF01C0EAFFEECF9A
:0C0B9C0000F00052E5E1006A016A12005E
:100BA8000A6A0350D8A40A800750D8A40A820A50B7
:100BB800D8B437EF06F0030AD8B4F0EF05F00AB05E
:100BC800EBEF05F006AE35EF06F033EF06F002AEB8
:100BD80033EF06F035EF06F00250800B0A6E029EE6
:100BE8000650800B069E0A18D8B401EF06F00A508A
:100BF800D8B433EF06F035EF06F00750035CD8B4ED
:100C08000BEF06F0D8A027EF06F02DEF06F0065000
:100C1800025CD8B415EF06F0D8A027EF06F02DEF48
:100C280006F00550015CD8B41FEF06F0D8A027EFF6
:100C380006F02DEF06F00450005CD8B437EF06F04C
:100C4800D8B02DEF06F00A52D8B435EF06F033EFDE
:100C580006F00A52D8B433EF06F035EF06F0D88024
:0E0C68001200D8901200D880D884120012001A
:0E0C7600A8B202D00000FCD724C3A9FF1200D0
:100C840024C302F025C303F002C000F003C001F046
:100C9400024A032A00C0E9FF01C0EAFFEE5201E064
:100CA400F3D703012451025C006E25510358016EF1
:0A0CB400010E005E000E015A12004E
:100CBE0028C300F003012807005228E024C3E9FFEF
:100CCE0025C3EAFFEE50000A0CE024C3E9FF25C35A
:100CDE00EAFF26C3D9FF27C3DAFFEE50DE1801E183
:100CEE000FD024C3E9FF25C3EAFF26C3D9FF27C3CC
:100CFE00DAFFDE50EE5C006E016A000E015A08D07B
:100D0E000301244B252B264B272BD2D7006A016AD1
:020D1E001200C1
:080D2000067EF0EC01F0120068
:100D28000B6A0350D8B4DAEF06F002500A6E028E4E
:100D38008E0E035E03AEDEEF06F0036C080E035C56
:100D4800D8A0B9EF06F0036E013602C001F0026ABE
:100D5800080E035CD8A0B9EF06F0036E0136016AED
:100D68000350D8A4D890C3EF06F00350D8B4C3EF0B
:100D780006F0D89002320132032EBDEF06F00BBC0C
:100D880001A0D0EF06F0D8A0D0EF06F0012AD8B421
:100D9800022A02BEEDEF06F00AAEF3EF06F0021EDD
:100DA800011E012AD8B4022AF3EF06F0026A016A8A
:100DB800F3EF06F00B800BAEF7EF06F0026A0AAE0F
:100DC800F7EF06F0FF0E026E016E0A360232F7EFF9
:100DD80006F0010E0C6EE2EC01F0F9EF06F0000EE1
:100DE8000C6EF9EF06F0FF0E0C6E0150006E02500B
:040DF800016E120076
:100DFC0000C008F00150006E016A026A036A0B6AB7
:100E0C000C6A016A026A036A960E036E0A6A00AEE5
:100E1C0016EF07F0081E001E082AD8B4002A0A8E06
:100E2C0000C001F008C000F0086A026AE3DC12009E
:100E3C000DC3F6FF0EC3F7FF0FC3F8FF0900F5CF84
:100E4C0000F0005211E00DC3F6FF0EC3F7FF0FC305
:100E5C00F8FF0900F5CF24F308DF010E03010D277D
:0A0E6C00000E0E230F23E4D712003E
:100E76000D0E0301246F4EDE0A0E0301246F4ADEB7
:020E8600120058
:100E88000301116B050E115D0AE211510F25E16E88
:100E9800000E1021E26E200EE66E112BF3D71151D1
:100EA8000F25E16E000E1021E26EE66A110711515E
:100EB8000F25126F000E1021136F0A0E046E000E1C
:100EC800056E0DC300F00EC301F02ADE08C000F065
:100ED80009C001F0300E002612C3E1FF13C3E2FF80
:100EE80000C0E6FF0A0E046E000E056E0DC300F08A
:100EF8000EC301F015DE00C00DF301C00EF3000EA5
:100F0800011802E1000E001801E102D01107CFD745
:020F18001200C5
:100F1A0003011351000805E3070E146F000E156F45
:100F2A0012D01351160805E2170E166F000E176F2E
:100F3A0006D01351010F166F176B000E172316C335
:100F4A0014F317C315F314C31EF315C31FF3186B59
:100F5A00196B046A056A066A076A0DC300F00EC3B4
:100F6A0001F00FC302F010C303F019DE010ED8B06E
:100F7A00000E006E005209E011C3E1FF12C3E2FF46
:100F8A002D0EE66E114B122B0F7F0DC304F00EC30C
:100F9A0005F00FC306F010C307F0006A016A026A7F
:100FAA00036AFDDD010ED8B0000E006E005235E076
:100FBA00000E046E000E056E000E066E7F0E076EA2
:100FCA000DC300F00EC301F00FC302F010C303F00B
:100FDA00E6DD010ED8B0000E006E00521EE00DC311
:100FEA0000F00EC301F00FC302F010C303F0000EAD
:100FFA00046E000E056E200E066E820E076EF5DC7C
:10100A0000C00DF301C00EF302C00FF303C010F3CA
:10101A00010E185F000E195BCBD7000E046E000E8E
:10102A00056E200E066E820E076E0DC300F00EC30B
:10103A0001F00FC302F010C303F0B1DD000ED8B007
:10104A00010E006E00521DE0000E046E000E056EC9
:10105A00200E066E820E076E0DC300F00EC301F05D
:10106A000FC302F010C303F003DC00C00DF301C08C
:10107A000EF302C00FF303C010F30301184B192B30
:10108A00CCD718511E2719511F23010E1A6F000EB3
:10109A001B6F010E006E000E016EABDE00C020F366
:1010AA0001C021F302C022F303C023F3800E1B19EF
:1010BA00006E800E1F19005C02E11E511A5D1EE2CD
:1010CA00000E046E000E056E200E066E820E076E6E
:1010DA0020C300F021C301F022C302F023C303F0AE
:1010EA003DEC04F000C020F301C021F302C022F35A
:1010FA0003C023F303011A4B1B2BD8D7000E046E2F
:10110A00000E056E000E066E800E076E20C300F0FC
:10111A0021C301F022C302F023C303F03DEC04F023
:10112A000DC304F00EC305F00FC306F010C307F099
:10113A00F0EC01F000C00DF301C00EF302C00FF392
:10114A0003C010F3000E046E000E056E200E066E2C
:10115A00820E076E24DD000ED8B0010E006E00521A
:10116A000BE0000E03010D6F000E0E6F000E0F6FE5
:10117A007F0E106F184B192B0301800E1919006E80
:10118A00800E005C02E1000E185D38E211C3E1FF37
:10119A0012C3E2FF300EE66E114B122B11C3E1FFB0
:1011AA0012C3E2FF2E0EE66E114B122B800E1F1990
:1011BA00006E800E005C02E1000E1E5D04E21E510C
:1011CA00185F1F51195BFF0E1A6FFF0E1B6F800EFF
:1011DA001919006E800E1B19005C02E11A51185D84
:1011EA000DE211C3E1FF12C3E2FF300EE66E114BAE
:1011FA00122B010E1A5F000E1B5BE9D71A6B1B6BD1
:10120A00800E1B19006E800E1F19005C02E11E5130
:10121A001A5D60E20DC300F00EC301F00FC302F0C5
:10122A0010C303F07CDD00C01CF301C01DF3300EB7
:10123A00002611C3E1FF12C3E2FF00C0E6FF114B13
:10124A00122B1B51191902E118511A1908E111C37D
:10125A00E1FF12C3E2FF2E0EE66E114B122B1CC3E6
:10126A0000F01DC301F0C5DD00C020F301C021F369
:10127A0002C022F303C023F300C004F001C005F04A
:10128A0002C006F003C007F00DC300F00EC301F060
:10129A000FC302F010C303F03EDD00C00DF301C01E
:1012AA000EF302C00FF303C010F3000E046E000E1B
:1012BA00056E200E066E820E076EFAEC04F000C070
:1012CA000DF301C00EF302C00FF303C010F31A4B63
:1012DA001B2B96D711C3E1FF12C3E2FFE66A120085
:1012EA000301106B0DC3E9FF0EC3EAFFEECF0FF344
:1012FA000F51000A0EE00FC324F30ADC0301102B7E
:10130A0010510D25E96E000E0E21EA6EEECF0FF395
:04131A00EFD71200F7
:10131E00220E0C6E086A096A0A6A0B6A0C06D8B4A9
:10132E001FD0D8900B320A32093208320332023201
:10133E0001320032D8A0F2D70C06D8B409D004502E
:10134E0008260550092206500A2207500B22EAD71A
:10135E00045008260550092206500A2207500B2277
:02136E0012006B
:10137000000E03010E1902E1000E0D1935E00DC338
:10138000E9FF0EC3EAFFEE522FE00FC324F310C3B0
:1013900025F378DC00C028F30DC324F30EC325F336
:1013A0000FC326F310C327F38ADC000E011802E1F5
:1013B000000E001805E10DC300F00EC301F016D0B9
:1013C000010E03010D25246F000E0E21256F0FC3A2
:1013D000E9FF10C3EAFFEECF26F3B6EC05F000C03C
:0E13E0000DF301C00EF3C4D7006A016A1200BB
:1013EE000201DF6BE06B000EE05D02E1800EDF5D5F
:1013FE000AE25F0EDF25E16E020EE021E26EE66A82
:10140E00DF4BE02BF0D70001936B946B916B926BDB
:10141E00AACF2CF202012C6B00018F6B906BA38A6A
:02142E001200AA
:101430000DC3F6FF0EC3F7FF0FC3F8FF0900F5CF8A
:1014400000F0005212E00DC3F6FF0EC3F7FF0FC30A
:10145000F8FF0900F5CF24F38DEC05F0010E030130
:0C1460000D27000E0E230F23E3D712000F
:10146C00C26A070EC16EC18E0DC300F0003600902B
:10147C00003600900050C212C280AFEC05F0C28260
:10148C00C2A201D0FDD7C4CF01F0006AC350001234
:08149C00000E0112C2901200C3
:1014A4000DC304F00EC305F004C0E9FF05C0EAFF54
:1014B400EE5203E0044A052AF7D704C002F005C03F
:1014C40003F0044A052A0FC300F010C301F003011E
:1014D4000F4B102B00C0E9FF01C0EAFF02C0E1FF7F
:1014E40003C0E2FFEECFE6FF02C0E9FF03C0EAFF5C
:1014F400EE5201E0E2D70DC300F00EC301F012007A
:101504000050086E0150006E016A026A036A0B6A99
:101514000C6A960E036E0A6A00C001F008C000F05F
:0A152400086A026A00EC04F01200ED
:10152E000301106B0DC3E9FF0EC3EAFFEECF0FF3FD
:10153E000F51000A0FE00FC324F33BEC06F003013A
:10154E00102B10510D25E96E000E0E21EA6EEECF16
:06155E000FF3EED71200AE
:101564000FC3F6FF10C3F7FF11C3F8FF0900F5CF4F
:1015740000F0005218E00FC3F6FF10C3F7FF11C3C9
:10158400F8FF0900F5CF00F00DC3E1FF0EC3E2FF41
:1015940000C0E6FF03010D4B0E2B010E0F27000EBA
:1015A40010231123DDD70DC3E1FF0EC3E2FFE66A6A
:0215B400120023
:1015B600C088F90EC16EFF0EC26EC098FF0E986EFF
:1015C600EF0E926EBF0E946E9396959692809594BA
:1015D60098869386959692988988958E99869598F9
:0815E60096988C988D98120074
:1015EE008C88100E0B6E390E0C6E0D0E0D6E0D2EB0
:1015FE00FED70C2EFCD70B2EFAD7000000008C98CD
:10160E00100E0B6E390E0C6E0D0E0D6E0D2EFED7CE
:10161E000C2EFCD70B2EFAD7000000008C88100E73
:10162E000B6E390E0C6E0D0E0D6E0D2EFED70C2E92
:0E163E00FCD70B2EFAD7000000008C9812008B
:10164C000201E36BE46B196A1A6A6F0E03010D6FEA
:10165C00340E0E6F000E0F6FE5DEC3DEFA0E0301C3
:10166C000D6F350E0E6F000E0F6F1EEC07F03D0E5A
:10167C000B6EE10E0C6E3F0E0D6E0D2EFED70C2E6A
:10168C00FCD70B2EFAD700000000000E00019019B9
:10169C0002E1010E8F1921E15F0E03010D6F020EA5
:1016AC000E6F3F0E0F6F000E106F5CDE000E026EA1
:1016BC000150025C02E1005000080FE2150E02011D
:1016CC00E36F000EE46F010E196E000E1A6E5F0EC2
:1016DC0003010D6F020E0E6F02DE1F0E0B6E710EEC
:1016EC000C6E1E0E0D6E0D2EFED70C2EFCD70B2E77
:1016FC00FAD700000201E34BE42B800EE419006ED4
:10170C00800E005C02E1140EE35D07E2000E1A1875
:0C171C0002E1000E191801E1A0D7120034
:101728008C988D98100E0B6E390E0C6E0D0E0D6E7A
:101738000D2EFED70C2EFCD70B2EFAD7000000007A
:101748008C88100E0B6E390E0C6E0D0E0D6E0D2E54
:10175800FED70C2EFCD70B2EFAD7000000008C9871
:101768008D88100E0B6E390E0C6E0D0E0D6E0D2E33
:10177800FED70C2EFCD70B2EFAD7000000008C8861
:101788008D98100E0B6E390E0C6E0D0E0D6E0D2E03
:10179800FED70C2EFCD70B2EFAD7000000008C9831
:0417A8008D98120006
:1017AC00AFCF01F0ACA202D0AC98AC8801C000F075
:0217BC00120019
:1017BE000900F5CFE6FF0006FBE10106F9E1120094
:1017CE001A0E0201266F0B0E276F240E286F030EC2
:1017DE00296FAC0E1E6F170E1F6F000E206F000EBE
:1017EE00216FFF0E166FFF0E176F000E186F000E93
:1017FE00196FFF0E1A6FFF0E1B6F000E1C6F000E7F
:10180E001D6FAD8A900EAC6E948E949C9EAA03D0E2
:08181E00AFCF00F0FBD7120070
:10182600760E0201266F0C0E276F240E286F030E0C
:10183600296FFF0E1E6FFF0E1F6F000E206F000E2A
:10184600216FFF0E166FFF0E176F000E186F000E3A
:10185600196FFF0E1A6FFF0E1B6F000E1C6F000E26
:101866001D6FA88A900E9C6E98849892A4AA03D0A5
:08187600AACF00F0FBD712001D
:10187E00FF0E0201226FFF0E236FFF0E246FFF0E6D
:0E188E00256FC26A070EC16EC18EC2801200A5
:10189C00C80E00019525E16E000E9621E26EE66AF7
:1018AC003A6A3B6A956B966BAFCF3CF03C6A3D6AEB
:0618BC003E6A9D8A120045
:1018C200C70E03010D6F320E0E6F000E0F6FAFDDEC
:1018D200E3C20DF3E4C20EF307DD3BEC07F086DD55
:1018E200220E03010D6F330E0E6F000E0F6F9FDD80
:1018F2000F0E006E000E016E026E036E5DC204F0EA
:101902005EC205F0000E02015EBFFF0E066E076E9C
:1019120005DD990E002403010D6F300E01200E6FBC
:10192200000E02200F6F83DD3BEC07F02D0E03014A
:101932000D6F020E0E6F810E0F6F350E106F000EBF
:10194200116F0FDE350E03010D6F020E0E6F0F0EBB
:10195200006E000E016E026E036E5DC204F05EC286
:1019620005F0000E02015EBFFF0E066E076ED6DCAA
:10197200990E002403010F6F300E0120106F000E2C
:101982000220116FEEDD2D0E03010D6F020E0E6FA0
:10199200CDDD0D0E246F3BEC06F0B70E0B6EA10EE3
:1019A2000C6EC30E0D6E0D2EFED70C2EFCD70B2E19
:1019B200FAD7000000005F0E03010D6F020E0E6FDA
:1019C20093DC3E0E02015F6F11DD3C0E03010D6FD1
:1019D200330E0E6F000E0F6F2ADDE1C20DF3E2C26D
:1019E2000EF3A4DD0D0E246F3BEC06F00A0E03018C
:1019F200246F3BEC06F01A0E0301246F3BEC06F059
:101A0200F5DC990E0B6E310E0C6EA20E0D6E0D2EC4
:101A1200FED70C2EFCD70B2EFAD700005F0E030167
:101A22000D6F020E0E6F60DC3BEC07F0DFDC120084
:101A3200E3C204F0E4C205F00201E751E81124E038
:101A4200010EE75F000EE85B04C002F005C003F080
:101A5200044A052AE5C200F0E6C201F0E54BE62B96
:101A620000C0E9FF01C0EAFF02C0E1FF03C0E2FFDC
:101A7200EECFE6FF02C0E9FF03C0EAFFEECF00F0BF
:101A8200005201E101D0D8D7E7C200F0E8C201F06C
:101A9200010EE75F000EE85B0050011008E004C091
:101AA200E1FF05C0E2FFE66A044A052AEDD7E3C278
:081AB20000F0E4C201F0120093
:101ABA0099DCE3C20DF3E4C20EF3E5C20FF31EECA8
:101ACA0007F0990E0B6E310E0C6EA20E0D6E0D2ED6
:101ADA00FED70C2EFCD70B2EFAD700005F0E03019F
:101AEA000D6F020E0E6F75EC09F00201E65336E037
:101AFA00090E0301246F8DEC05F05F0E03010D6FD3
:101B0A00020E0E6F420E0F6F000E106F2CDC000ECD
:101B1A00026E0150025C02E10050000803E200017B
:101B2A00C64BC72B2E0E03010D6F350E0E6F000E1E
:101B3A000F6F79DCC6C00DF3C7C00EF3E1C20FF315
:101B4A00E2C210F344EC07F0E1C20DF3E2C20EF375
:101B5A0075EC09F0090E246F8DEC05F03BEC07F0EB
:021B6A00120067
:101B6C00D596D584D582D580D59AD59C480ED76E7E
:101B7C00E50ED66EF2940201126B136B146B156B9F
:081B8C00F184F28AD58E1200EB
:101B9400E3C2E1FFE4C2E2FFE66AE3C20DF3E4C29A
:101BA4000EF32D0E03010F6F340E106F000E116F24
:101BB400D7DCE3C224F3E4C225F342EC06F000C010
:101BC40095F001C096F00201E56BE50E03010D6F7F
:101BD400020E0E6F9B0E0F6F350E106F000E116FFD
:101BE400BFDCE50E0301246F020E256F42EC06F004
:101BF40000C095F001C096F0E50E0024E16E020EDF
:101C04000120E26E006A83BE002A300E002600C066
:101C1400E6FF0001954B962BE50E9525E16E020E2D
:101C24009621E26E0D0EE66E0201DF4BE02BE50E0F
:101C340000019525E16E020E9621E26E0A0EE66E13
:101C44000201DF4BE02BE50E00019525E16E020E4B
:101C54009621E26EE66AE3C20DF3E4C20EF3E50EEA
:101C640003010F6F020E106F1BDC0201E56BE50E22
:101C740003010D6F020E0E6F930E0F6F350E106F72
:101C8400000E116F6DDCE50E0301246F020E256F4B
:101C940042EC06F000C095F001C096F0E50E002479
:101CA400E16E020E0120E26E006A87B6002A300E51
:101CB400002600C0E6FF0001954B962BE50E952506
:101CC400E16E020E9621E26E0D0EE66E954B962B9A
:101CD400E50E9525E16E020E9621E26E0A0EE66E81
:101CE400954B962BE50E9525E16E020E9621E26E3C
:101CF400E66AE3C20DF3E4C20EF3E50E03010F6FCF
:101D0400020E106F52EC0AF00201E56BE50E0301BE
:101D14000D6F020E0E6FB30E0F6F350E106F000EA7
:101D2400116F1EDCE50E0301246F020E256F42ECD9
:101D340006F000C095F001C096F0E50E0024E16EB7
:101D4400020E0120E26E006A83B8002A300E0026DB
:101D540000C0E6FF0001954B962BE50E9525E16E3C
:101D6400020E9621E26E0D0EE66E954B962BE50E55
:101D74009525E16E020E9621E26E0A0EE66E954BF3
:101D8400962BE50E9525E16E020E9621E26EE66A2B
:101D9400E3C20DF3E4C20EF3E50E03010F6F020E6E
:101DA400106F52EC0AF00201E56BE50E03010D6FB2
:101DB400020E0E6FAB0E0F6F350E106F000E116F0B
:101DC400B2EC0AF0E50E0301246F020E256F42EC1B
:101DD40006F000C095F001C096F0E50E0024E16E17
:101DE400020E0120E26E006A84B8002A300E00263A
:101DF40000C0E6FF0001954B962BE50E9525E16E9C
:101E0400020E9621E26E0D0EE66E954B962BE50EB4
:101E14009525E16E020E9621E26E0A0EE66E954B52
:101E2400962BE50E9525E16E020E9621E26EE66A8A
:101E3400E3C20DF3E4C20EF3E50E03010F6F020ECD
:101E4400106F52EC0AF00201E56B010E03010D6FF5
:101E540036EC0AF000C02AF201C02BF2E50E0301B1
:101E64000D6F020E0E6FC20E0F6F350E106F000E47
:101E7400116FB2EC0AF0E50E0301246F020E256F18
:101E840042EC06F000C095F001C096F02AC20DF3B2
:101E94002BC20EF3E50E00240F6F020E0120106F0B
:101EA40044EC07F0E50E246F020E256F42EC06F0B9
:101EB40000C095F001C096F0E50E0024E16E020E1C
:101EC4000120E26E0D0EE66E0001954B962BE50E99
:101ED4009525E16E020E9621E26E0A0EE66E954B92
:101EE400962BE50E9525E16E020E9621E26EE66ACA
:101EF400E3C20DF3E4C20EF3E50E03010F6F020E0D
:101F0400106F52EC0AF00201E56B020E03010D6F33
:101F140036EC0AF0060E005C0101486F000E015811
:101F2400496FE50E03010D6F020E0E6FA30E0F6FC6
:101F3400350E106F000E116FB2EC0AF0E50E0301BE
:101F4400246F020E256F42EC06F000C095F001C02C
:101F540096F048C100F049C101F082EC0AF0000E8D
:101F6400046E000E056E250E066E870E076EFAECE3
:101F740004F0000E046E000E056E000E066E890E4F
:101F8400076E3DEC04F000C04AF101C04BF102C001
:101F94004CF103C04DF100C00DF301C00EF302C0BB
:101FA4000FF303C010F3E50E000195250301116F33
:101FB400020E000196210301126F020E136F8DECC5
:101FC40007F0E50E246F020E256F42EC06F000C008
:101FD40095F001C096F0E50E0024E16E020E01209A
:101FE400E26EB00EE66E0001954B962BE50E95253C
:101FF400E16E020E9621E26E430EE66E954B962B31
:10200400E50E9525E16E020E9621E26EE66AE3C2C4
:102014000DF3E4C20EF3E50E03010F6F020E106F11
:1020240052EC0AF00201E56BE50E03010D6F020E9E
:102034000E6F6E0E0F6F350E106F000E116FB2EC37
:102044000AF0E3C20DF3E4C20EF3E50E03010F6FD1
:10205400020E106F52EC0AF0E3C224F3E4C225F33B
:0E20640042EC06F000C095F001C096F01200AC
:10207200FFEC1AF0DBEC0AF094EC0BF0920E02018A
:10208200E16F010EE26F0101926B526B02015F6B15
:102092002A6B2B6B01014E6B4F6B506B516B000126
:1020A200C66BC76B9D879D9502015D6B5E6B7E86DD
:1020B200020E7F6E700EB06EAD84E7EC0BF00C0E6C
:1020C2000301246F8DEC05F01F0E0B6E710E0C6E6A
:1020D2001E0E0D6E0D2EFED70C2EFCD70B2EFAD730
:1020E20000003BEC07F0690E03010D6F320E0E6F1C
:1020F200000E0F6F18EC0AF06C0E03010D6F300E1C
:102102000E6F000E0F6F18EC0AF0DB0E03010D6F5D
:102112002F0E0E6F000E0F6F18EC0AF0F7EC0AF09C
:102122007C86020E7D6E700EAB6EA88413EC0CF0F2
:10213200380E03010D6F2F0E0E6F000E0F6F18EC8D
:102142000AF03D0E0B6EE10E0C6E3F0E0D6E0D2E63
:10215200FED70C2EFCD70B2EFAD7000000008C8481
:10216200020E0A6E310E0B6E620E0C6E450E0D6E75
:102172000D2EFED70C2EFCD70B2EFAD70A2EF8D72F
:102182008C943D0E0B6EE10E0C6E3F0E0D6E0D2EFD
:10219200FED70C2EFCD70B2EFAD7000000008C962F
:1021A200D30E03010D6F330E0E6F000E0F6F18EC7E
:1021B2000AF0F7EC09F0AC8ED08E9E9AA38AF28CCC
:1021C200F28E26EC0BF0000E1A1802E1010E19181D
:1021D2000AE1BE0E03010D6F340E0E6F000E0F6F7B
:1021E20018EC0AF019D0E60E03010D6F320E0E6FD5
:1021F200000E0F6F18EC0AF08C783D0E0B6EE10E9C
:102202000C6E3F0E0D6E0D2EFED70C2EFCD70B2E34
:10221200FAD700000000F0D73FEC0CF0E10E03010A
:102222000D6F310E0E6F000E0F6F18EC0AF0010EDB
:1022320003010D6F36EC0AF000C02AF201C02BF246
:1022420000C00DF301C00EF3E1C20FF3E2C210F3BE
:1022520044EC07F0E1C20DF3E2C20EF375EC09F0B3
:10226200090E246F8DEC05F0020E03010D6F36ECA2
:102272000AF000C048F101C049F100C00DF301C0ED
:102282000EF3E1C20FF3E2C210F344EC07F0E1C235
:102292000DF3E2C20EF375EC09F03BEC07F0920E7F
:1022A2000201E16F010EE26F050E03010D6F320EA6
:1022B2000E6F000E0F6F18EC0AF0E1C2E3F2E2C2F9
:1022C200E4F267DC00C09BF001C09CF03BEC07F03D
:1022D200070E0B6E170E0C6E6A0E0D6E0D2EFED7CC
:1022E2000C2EFCD70B2EFAD70000750E03010D6FD2
:1022F2002F0E0E6F000E0F6F18EC0AF00001C66B66
:10230200C76B9D87890E03010D6F320E0E6F000E93
:102312000F6F18EC0AF0EF0E0201E36F340EE46F58
:10232200000EE56F000E00019DB7010E0201E66F7F
:102332005DEC0DF0C60E03010D6F300E0E6F000E38
:102342000F6F18EC0AF0450E0201E36F350EE46FD1
:10235200000EE56F000E00019DB7010E0201E66F4F
:102362005DEC0DF06C0E03010D6F310E0E6F000E61
:102372000F6F18EC0AF00A0E0201E36F350EE46FDC
:10238200000EE56F000E00019DB7010E0201E66F1F
:102392005DEC0DF0A80E03010D6F320E0E6F000EF4
:1023A2000F6F18EC0AF05A0E0201E36F350EE46F5C
:1023B200000EE56F000E00019DB7010E0201E66FEF
:1023C2005DEC0DF0280E03010D6F320E0E6F000E44
:1023D2000F6F18EC0AF0780E0201E36F350EE46F0E
:1023E200000EE56F000E00019DB7010E0201E66FBF
:1023F2005DEC0DF01A0E03010D6F310E0E6F000E23
:102402000F6F18EC0AF0EE0E0201E36F350EE46F67
:10241200000EE56F000E00019DB7010E0201E66F8E
:102422005DEC0DF0BA0E03010D6F310E0E6F000E52
:102432000F6F18EC0AF0A30E0201E36F330EE46F84
:10244200000EE56F000E00019DB7010E0201E66F5E
:102452005DEC0DF0F00E03010D6F300E0E6F000EED
:102462000F6F18EC0AF0FD0E0201E36F340EE46FF9
:10247200000EE56F000E00019DB7010E0201E66F2E
:102482005DEC0DF00D0E03010D6F300E0E6F000EA0
:102492000F6F18EC0AF0500E0201E36F350EE46F75
:1024A200000EE56F000E00019DB7010E0201E66FFE
:1024B2005DEC0DF0930E03010D6F310E0E6F000EE9
:1024C2000F6F18EC0AF0640E0201E36F350EE46F31
:1024D200000EE56F000E00019DB7010E0201E66FCE
:1024E2005DEC0DF0BB0E03010D6F330E0E6F000E8F
:1024F2000F6F18EC0AF0D60E0201E36F350EE46F8F
:10250200000EE56F000E00019DB7010E0201E66F9D
:102512005DEC0DF0430E03010D6F310E0E6F000ED8
:102522000F6F18EC0AF0E00E0201E36F340EE46F55
:10253200000EE56F000E00019DB7010E0201E66F6D
:102542005DEC0DF0AC0E03010D6F340E0E6F000E3C
:102552000F6F18EC0AF0C6C00DF3C7C00EF3E1C24C
:102562000FF3E2C210F344EC07F0E1C20DF3E2C252
:102572000EF375EC09F03A0E0D6F350E0E6F000E6C
:102582000F6F18EC0AF0000E0001C71902E10C0EE1
:10259200C6190CE1DC0E03010D6F350E0E6F000E35
:1025A2000F6F18EC0AF000019D850BD0C90E0301D4
:1025B2000D6F350E0E6F000E0F6F18EC0AF0000152
:1025C2009D953BEC07F00001C66BC76B9D97EA0E29
:1025D20003010D6F330E0E6F000E0F6F18EC0AF031
:1025E2004EEC0CF09E9A9D8A976B986B000E01013F
:1025F200511902E1000E5019D8A40DD197C00DF364
:1026020098C00EF3520E03010F6F010E106F44ECCF
:1026120007F0520E0D6F010E0E6F75EC09F0010EF0
:102622000D6F36EC0AF000C02AF201C02BF200C096
:102632000DF301C00EF3520E03010F6F010E106F66
:1026420044EC07F0170E0D6F340E0E6F000E0F6F75
:1026520018EC0AF0520E03010D6F010E0E6F75ECAD
:1026620009F0D00E0D6F350E0E6F000E0F6F18ECC5
:102672000AF0020E03010D6F36EC0AF0060E005E40
:10268200000E015A00C048F101C049F100C00DF32B
:1026920001C00EF3520E03010F6F010E106F44ECD6
:1026A20007F0520E0D6F010E0E6F75EC09F0160E4B
:1026B2000D6F350E0E6F000E0F6F18EC0AF048C149
:1026C20000F049C101F082EC0AF0000E046E000E27
:1026D200056E250E066E870E076EFAEC04F0000EEC
:1026E200046E000E056E000E066E890E076E3DEC3E
:1026F20004F000C04AF101C04BF102C04CF103C02A
:102702004DF100C00DF301C00EF302C00FF303C080
:1027120010F3520E0301116F010E126F020E136FAE
:102722008DEC07F0520E0D6F010E0E6F75EC09F075
:10273200220E0D6F350E0E6F000E0F6F18EC0AF0A1
:10274200000E83BE010E0301246F300E24278DEC90
:1027520005F0E20E03010D6F350E0E6F000E0F6FC6
:1027620018EC0AF0000E87B6010E0301246F300E3A
:1027720024278DEC05F0F40E03010D6F350E0E6F5C
:10278200000E0F6F18EC0AF0000E83B8010E030161
:10279200246F300E24278DEC05F0E80E03010D6F37
:1027A200350E0E6F000E0F6F18EC0AF0000E84B893
:1027B200010E0301246F300E24278DEC05F08A0EE2
:1027C20003010D6F350E0E6F000E0F6F18EC0AF03D
:1027D200000E00019DB5010E0301246F300E242767
:1027E2008DEC05F0BB0E03010D6F350E0E6F000E62
:1027F2000F6F18EC0AF0000E80B0010E0301246F77
:10280200300E24278DEC05F03B0E0301246F8DEC76
:1028120005F03BEC07F002012B51020802E12A51BC
:10282200000808E3000E0101495D02E13E0E485D29
:1028320001E31FD00101000E4F1902E1000E4E19F3
:1028420018E100019DA515D0010E01014E6F000E89
:102852004F6FE1C2E3F2E2C2E4F2CAEC0DF000C053
:102862009BF001C09CF0E1C2E3F2E2C2E4F261EC4F
:102872000CF00001000E901902E1010E8F19D8A48C
:1028820079D25F0E03010D6F020E0E6F300E0F6FC5
:10289200000E106FB8EC09F000C099F001C09AF078
:1028A200000E026E0150025C02E1005000082AE2B2
:1028B200F7EC09F03D0E03010D6F300E0E6F000EA6
:1028C2000F6F18EC0AF0010E03010D6F340E0E6F3C
:1028D200000E0F6F1EEC07F0D60E0B6E110E0C6E73
:1028E200E40E0D6E0D2EFED70C2EFCD70B2EFAD752
:1028F20000005F0E03010D6F020E0E6F75EC09F002
:102902003BEC07F05F0E03010D6F020E0E6F350EEA
:102912000F6F000E106FB8EC09F000C099F001C003
:102922009AF0000E026E0150025C02E100500008B3
:1029320055E29E0E03010D6F000E0E6F490E0F6FD2
:10294200320E106F000E116FB2EC0AF0A70E0201E8
:10295200E36F000EE46F040E000199250201E56F9A
:10296200000E00019A210201E66F0E0EE76F000EC3
:10297200E86F19EC0DF0980E03010D6F340E0E6F17
:10298200000E0F6F18EC0AF09E0E03010D6F000E81
:102992000E6F75EC09F03BEC07F0F7EC09F09E0EB8
:1029A20003010D6F000E0E6F97EC0AF0B70E0B6E5F
:1029B200A10E0C6EC30E0D6E0D2EFED70C2EFCD783
:1029C2000B2EFAD7000000005F0E0D6F020E0E6F85
:1029D20075EC09F03BEC07F0F7EC09F05F0E030130
:1029E2000D6F020E0E6F1B0E0F6F000E106FB8EC04
:1029F20009F000C099F001C09AF0000E026E015079
:102A0200025C02E1005000080DE200019D95430EB8
:102A120003010D6F340E0E6F000E0F6F18EC0AF0EB
:102A2200F7EC09F05F0E03010D6F020E0E6F260E1A
:102A32000F6F000E106FB8EC09F000C099F001C0E2
:102A42009AF0000E026E0150025C02E10050000892
:102A52000DE200019D85560E03010D6F330E0E6FC0
:102A6200000E0F6F18EC0AF0F7EC09F05F0E03018D
:102A72000D6F020E0E6F630E0F6F000E106FB8EC2B
:102A820009F000C099F001C09AF0000E026E0150E8
:102A9200025C02E1005000084EE2700E03010D6F6D
:102AA200330E0E6F000E0F6F18EC0AF0E1C2E3F264
:102AB200E2C2E4F2CAEC0DF000C09BF001C09CF04F
:102AC200020E02015D6F000E5E6F5F0E03010D6F5D
:102AD200020E0E6F720E0F6F000E106FB8EC09F03F
:102AE200000E026E0150025C02E10050000803E297
:102AF20002015D6B5E6B5F0E03010D6F020E0E6FC6
:102B02005E0E0F6F000E106FB8EC09F0000E026E31
:102B12000150025C02E10050000805E2010E0201D0
:102B22005D6F000E5E6FE1C2E3F2E2C2E4F261ECBD
:102B32000CF0F7EC09F05F0E03010D6F020E0E6F41
:102B4200520E0F6F000E106FB8EC09F000C099F032
:102B520001C09AF0000E026E0150025C02E10050C8
:102B62000008D8B0DFD0070E00019925E96E000EEB
:102B72009A21EA6EEE50310A30E15F0E03010D6FC9
:102B8200020E0E6F5A0E0F6F000E106FB8EC09F0A6
:102B920000C099F001C09AF0000E026E0150025C72
:102BA20002E100500008D8A08C88680E03010D6F66
:102BB200020E0E6F860E0F6F000E106FB8EC09F04A
:102BC20000C099F001C09AF0000E026E0150025C42
:102BD20002E100500008D8A08C98070E0001992548
:102BE200E96E000E9A21EA6EEE50320A30E15F0E73
:102BF20003010D6F020E0E6F8B0E0F6F000E106F22
:102C0200B8EC09F000C099F001C09AF0000E026E13
:102C12000150025C02E100500008D8A08D885F0ECE
:102C220003010D6F020E0E6F810E0F6F000E106FFB
:102C3200B8EC09F000C099F001C09AF0000E026EE3
:102C42000150025C02E100500008D8A08D98840E69
:102C520003010D6F340E0E6F000E0F6F18EC0AF0A9
:102C6200E1C20DF3E2C20EF38A0E03010F6F330EBF
:102C7200106F000E116FB2EC0AF00E0E0201E12588
:102C8200E16E000EE221E26E006A8CB8002A300E7C
:102C9200002600C0E6FF160EE125E16E000EE221DD
:102CA200E26E006A8DB8002A300E002600C0E6FFF0
:102CB200020E5D6F000E5E6F5F0E03010D6F020E5E
:102CC2000E6F770E0F6F000E106FB8EC09F0000E4A
:102CD200026E0150025C02E10050000803E20201B0
:102CE2005D6B5E6B5F0E03010D6F020E0E6F7C0E4D
:102CF2000F6F000E106FB8EC09F0000E026E01505B
:102D0200025C02E10050000805E2010E02015D6F63
:102D1200000E5E6FE1C2E3F2E2C2E4F261EC0CF09B
:102D2200F7EC09F0A80E03010D6F2F0E0E6F000EC7
:102D32000F6F18EC0AF0590E0201E36F340EE46FC4
:102D4200000EE56F000E00019DB7010E0201E66F55
:102D52005DEC0DF00D0E0B6E2D0E0C6ED70E0D6E82
:102D62000D2EFED70C2EFCD70B2EFAD7000000003A
:102D7200F7EC09F0974B982B800E006E800E981995
:102D8200005C02E197513B0806E201014E6B4F6B7A
:102D92000001976B986B000E901902E1020E8F19D9
:102DA2000BE1050E03010D6F330E0E6F000E0F6F58
:102DB20018EC0AF0F7EC09F0000E3E1802E1010EE1
:102DC2003D186AE1D00E03010D6F340E0E6F000E36
:102DD2000F6F18EC0AF0C80E03010D6F000E0E6F94
:102DE20075EC09F03BEC07F0C80E0301246F000EEE
:102DF200256F4C0E266F000E276F050E286F5FECB5
:102E020006F0000E011802E1000E001807E1010EA3
:102E12000101506F000E516F4EEC0CF0C80E030111
:102E2200246F000E256F450E266F000E276F060ECB
:102E3200286F5FEC06F0000E011802E1000E001888
:102E420005E10101506B516B4EEC0CF0C80E030111
:102E52000D6F000E0E6F97EC0AF00D0E246F3BEC17
:102E620006F0F7EC09F07A0E0B6EC10E0C6E810EB5
:102E72000D6E0D2EFED70C2EFCD70B2EFAD70000AE
:102E820000005F0E03010D6F020E0E6F75EC09F06C
:102E9200F7EC09F04EEC0CF0B6EC0DF0000E151943
:102EA20002E1000E141901E1F9D780B002D000014D
:082EB2009D95F7EF12F0FFD728
:1035FE0010EE19F07E0E006E010E016EBA0EF66E12
:0E360E002E0EF76E000EF86EDFEC0BF01200C1
:022EBA00000016
:0B2EBC00537572766579204F66660042
:0A2EC700537572766579204F6E0096
:052ED100434D544900CF
:052ED6004D41483D00E4
:022EDB000000F5
:012EDD0000F4
:022EDE000000F2
:032EE0004F4B0055
:032EE3004F4B0052
:072EE6004E6F726D616C007C
:062EED00446562756700F8
:082EF300436465204C65640096
:042EFB00204F6E00F6
:052EFF003338333700F9
:0F2F040044617461204F6E2044656D616E6400FE
:052F13003437313500E8
:052F18003437313500E3
:052F1D003338333700DA
:052F2200204F6666006F
:052F2700204F6666006A
:042F2C00204F6E00C4
:022F300000009F
:022F320000009D
:022F340000009B
:022F3600000099
:102F380020496E69742056425241592055415254D5
:102F4800312031393230302C382C4E2C31206574F8
:102F5800205155454354454C205541525432203157
:0D2F6800393230302C382C4E2C310D0A003F
:102F7500204C696169736F6E20646566696E696569
:102F850020706F7572205374617261646963742077
:102F95004949202B33333678787878787878352016
:032FA5000D0A0012
:102FA80045666661636520746F7573206C65732070
:102FB800534D53207265E77573202841542B514DAA
:102FC8004744413D2244454C20494E424F5822290E
:032FD8000D0A00DF
:102FDB002047534D325F636C69636B5F3138463802
:102FEB00374A35305F55617274315F556172743297
:102FFB005F55415254315F3135313030362E630DD0
:02300B000A00B9
:10300D00205465737420736920656E7265676973EA
:10301D007472E920737572206C6520726573656139
:10302D0075202841542B435245473F31290D0A0045
:10303D002052656164206D657373616765204E4F25
:10304D004E204C5553202841542B434D474C3D2287
:0F305D0052454320554E5245414422290D0A0049
:10306C002047534D322D636C69636B205465737428
:10307C00207769746820436C69636B6572322050E9
:0D308C00494331384638374A35300D0A00C7
:10309900222B333336323133333437313522002260
:1030A9002B333336313431333338333722004E6FD3
:0D30B9007420616666656374656400000044
:1030C6002053656E64204D736720747970652061A6
:1030D600732074657874206D6F6465202841542BC5
:0A30E600434D47463D31290D0A0015
:1030F0002052656E766F6920534D53207375722090
:103100007465726D696E616C202841542B434E4D7D
:0A311000493D322C3129200D0A0040
:10311A0020466F726D6174206465205265706F6E0F
:10312A00736520766961206C6962656C6CE9202898
:09313A004154563129200D0A0010
:10314300204C69737420616C6C206D736720667208
:103153006F6D20696E626F78202841542B434D4771
:093163004C3D414C4C290D0A00C1
:10316C00204E6576657220676F20696E20534C4542
:10317C004550206D6F64652841542B5153434C4B83
:07318C003D3029200D0A006F
:10319300204C656374757265206465206461746591
:1031A300206574206865757265202841542B43435C
:0731B3004C4B3F290D0A00FF
:1031BA002053656C65637420534D202841542B437A
:1031CA00504D533D22534D222C22534D222C225333
:0731DA004D2220200D0A0028
:1031E1002031657265204C656374757265204144B8
:1031F10043205241312065742041444320524132E1
:04320100200D0A0092
:10320500200D0A436F6E737469747574696F6E204F
:10321500647520534D5320E020656E766F79657295
:033225000D0A008F
:1032280020494D45492053657269616C206E756D62
:10323800626572202841542B4347534E29200D0ABA
:013248000085
:1032490041542B43434C4B3D2231352F30392F32DA
:10325900392C31363A34353A30302B3034220D009E
:103269002056657273696F6E203A205665727369CC
:103279006F6E2030362F31302F313520610D0A0025
:10328900205365742050494E20636F64652841546A
:0F3299002B4350494E3D3132333429200D0A006A
:1032A80020536F6674776172652056657273696F13
:0F32B8006E202841542B43474D5229200D0A0008
:1032C700200D0A20436F6E74656E75206475205358
:0F32D7004D5320E020656E766F7965720D0A0009
:1032E6002031393230302042617564207261746554
:0F32F600204E65676F636520424144200D0A003A
:10330500204465626F7264656D656E7420627566D2
:0D331500666572205541525432200D0A00A9
:1033220020436F6D706F7365204E756D65726F20EF
:0A3332002841542B434D47533D0042
:10333C00204F4B20706F757220656E766F69204D33
:0A334C00736720747874200D0A00E6
:10335600204469616C6F67756520534D5320726513
:0A3366007461626C6974200D0A00A6
:1033700020456E766F692044617461732064656DC9
:0A338000616E64E96573200D0A0018
:10338A000D5265746F7572204C6564313D2078204A
:09339A004C6564323D20780D0001
:1033A30041542B43504D533D22534D222C22534D18
:0833B300222C22534D220D00D3
:1033BB002053617665742070726F66696C65202886
:0833CB0041542657290D0A00A8
:1033D3002041726D65205258204954205541525462
:0733E30032202E2E0D0A001E
:1033EA002041726D6520525820495420554152544B
:0733FA0031202E2E0D0A0008
:1034010041542B434D474C3D2252454320554E528A
:06341100454144220D00BC
:10341700204D657375726520416E616C6F672E2054
:063427003B4541313D0070
:10342D000D0A47534D322050494331384638374AFB
:06343D0035303A0D0A00D3
:103443002053544F50206469616C6F677565205336
:063453004D53200D0A009C
:1034590041542B514D4744413D2244454C20494E4E
:06346900424F58220D0045
:10346F00204E65676F6365206261756420726174B9
:05347F0065200D0A00AC
:10348400205265746F757220636465204C656473A3
:04349400200D0A00FD
:10349800204D414A20646174652065742048657533
:0434A8007265200029
:1034AC00205068617365206427696E697420656EAD
:0234BC002000EE
:1034BE00204E65676F636520726575737369200DA5
:0234CE000A00F2
:1034D00020526563657074205541525431203A0082
:0F34E00041542B434D474C3D22414C4C220D0093
:0E34EF0041542B4350494E3D313233340D00D1
:0D34FD0041542B434E4D493D322C310D0002
:0C350A0041542B5153434C4B3D300D00FD
:0C3516003B736F69742054656D703D00BC
:0C3522003B20B04320203B4250313D00D4
:0C352E004C61737420537465703A2000E7
:0B353A0020706173202F203132200030
:0B35450041542B434D47463D310D0023
:0A35500041542B435245473F0D0044
:0A355A0041542B43474D520D0A0067
:0A35640041542B43434C4B3F0D0034
:0A356E000D0A20456E642E0D0A00C0
:0935780041542B4347534E0D0052
:0935810041542B434D47533D001A
:09358A003B4469616C6F673D0070
:0835930020425032203D2000CF
:08359B0020425031203D2000C8
:0835A3002054656D703D20000D
:0835AB00204C4432203D2000B9
:0835B300204C4431203D2000B2
:0735BB003B535441543D0055
:0735C200204541313D2000CE
:0735C9002E2E4241442100B7
:0635D0003B4541323D00C5
:0635D600415426570D00D0
:0635DC002E2E204F4B00D3
:0635E2003B4250323D00A7
:0635E8003B4C44323D00A3
:0635EE00415456310D00AE
:0635F4003B4C44313D0098
:0435FA0041540D002B
:020000040001F9
:06FFF800ACF705FFF0FF6D
:00000001FF
